:020000040000FA
:040000008A01002948
:08000800DD00030EDE00AD1C5B
:100010000C285708CF0022282D1C11285608CF0085
:100020002228AC1F16285508CF0022282C1F1B2879
:100030005408CF002228AC1E20285308CF002228C5
:100040000130CF0008080339C7004606031970289D
:10005000460D47060239C9004806031932284908E7
:10006000C80070284708C600C81C552834187028D6
:100070004F08AC07031C3D28AD0A5008AD072C08FB
:10008000DA002D08DB005A083902031CDB0A5B0882
:100090003A020318702834142C08B5002D08B60055
:1000A0003908AC003A08AD007028341C5C283508CB
:1000B000AC003608AD0034104F08D1005008D20013
:1000C000D109D209D10F6528D20A5108AC07031C07
:1000D0006A28AD0A5208AD07AD1F7028AC01AD010A
:1000E000AF1C75285708CF008B282F1C7A2856087C
:1000F000CF008B28AE1F7F285508CF008B282E1FDE
:1001000084285408CF008B28AE1E89285308CF00BE
:100110008B280130CF0008080C39CC004B06031D9A
:100120009228DA284B0D4C060839CE004D060319EB
:100130009C284E08CD00DA284C08CB00CD1DBF28E6
:10014000B418DA284F08AE07031CA728AF0A5008D6
:10015000AF072E08DA002F08DB005A083B02031C09
:10016000DB0A5B083C020318DA28B4142E08B70037
:100170002F08B8003B08AE003C08AF00DA28B41CDA
:10018000C6283708AE003808AF00B4104F08D100B9
:100190005008D200D109D209D10FCF28D20A510874
:1001A000AE07031CD428AF0A5208AF07AF1FDA28E6
:1001B000AE01AF010B115E0E8300DD0E5D0E090076
:100200008312031385018316031306309F00FF300A
:100210008500003086000F308700FF3088000030F6
:1002200089008113831203138501860187018801E8
:1002300089018C220130C400A000A100D001B924A2
:10024000AA24F624831203178D0183120313692451
:100250000C0883120313D30069240C0883120313C0
:10026000D40069240C0883120313D50069240C08F8
:1002700083120313D60069240C0883120313D700DA
:10028000E830B900BB000330BA00BC001430D9001C
:100290000808F039BD00F03A031D162BA424D90B31
:1002A0004829B024F82119224E24831603138030E4
:1002B0008100A0308B0083120313A424AC01AD0194
:1002C000AE01AF01B001B101B201B301B501B60198
:1002D000B701B8013410B4108B13421030082C064B
:1002E000031D421431082D06031D421432082E0648
:1002F000031D421433082F06031D42142C08B000BE
:100300002D08B1002E08B2002F08B3008B17C40BC4
:100310008C2919220A30C4000808F039BD00F03ACF
:10032000031D9521421CB7216C293D1E9A29BD1E33
:10033000A9290800A10A0310A00D10302002031DF6
:10034000A5290830A0000430A1004E24A123B72124
:100350000800A1030310A00C00302007031DB329DF
:100360000130A000A1004E24A123B7210800BF0145
:10037000C001C1012008BF00300EF039BF04300EAB
:100380000F39C000310E3039C00432184017B2188E
:10039000C0173208D900D90C590C3F39C1003318A5
:1003A0004117B318C1170910891009111830BE0080
:1003B000C10CC00CBF0C031CDF290914E029091073
:1003C000EF218914EF218910EF21BE0BD8290915DF
:1003D0000614EF210911EF210910061408008324E7
:1003E00008000330A90000000000A90BF329080051
:1003F00003101030A800A501A601A701A30DA40DAC
:10040000A50DA60DA70DA80B062A0800253084000F
:100410000E22840A0E22840A0E22FE2903300007CF
:10042000D900D91980001E300007D900D91B8000DF
:1004300008008030E4224330F8223D30F8223008B2
:10044000A3003108A400F82132228A30E4224C3083
:10045000F8223D30F8223208A3003308A400F82126
:1004600032220800DC01260E0F3903193A2A303EE9
:10047000F8223D2A5C162030F82226080F39031D89
:10048000472A5C1E472A2030F822DC15492A303ED4
:10049000F822250E0F39031D522ADC1D522A203066
:1004A000F822542A303EF82225080F39303EF8222F
:1004B00008003208A3003308A400F821DC018A30C8
:1004C000E4224C30F8223D30F822DC01260E0F39B0
:1004D00003196D2A303EF822702A5C162030F8226B
:1004E00026080F39031D7A2A5C1E7A2A2030F8224A
:1004F000DC157C2A303EF822250E0F39031D852A93
:10050000DC1D852A2030F822872A303EF822250873
:100510000F39303EF822080000308600A4240E2354
:100520000E2386150E230E23303086049824861160
:100530000E230E230030860086150E230E23303046
:100540008604832486110E230E2300308600861530
:100550000E230E2330308604832486110E230E23AF
:100560000030860086150E230E2320308604832457
:10057000861100308600C5222830E4220C30E422A7
:100580000630E4220130E422080083160313F03021
:1005900086008312031386100615000086150000DE
:1005A000861FD82A86110000861500008611CE2AE3
:1005B00086110000861500008611061183160313AC
:1005C0008601831203130800D900D800E922590ECE
:1005D000D800C5220030860086100E2306110E2397
:1005E00086150E235808F03986040E23861108005C
:1005F000D900D800FD22590ED800C522003086004F
:1006000086140E2306110E2386150E235808F03982
:1006100086040E2386110E238610080000000000B9
:100620000000000000000000000008002324AA24AD
:100630000808F039BD00F03A031D182BA424B0249B
:10064000B223BE23D4235308CF00A823A1237623AB
:100650004F08D300DF235408CF00A823A12376231B
:100660004F08D400EE235508CF00A823A1237623FA
:100670004F08D500FF235608CF00A823A1237623D7
:100680004F08D60010245708CF00A823A1237623B3
:100690004F08D700831203178D01831203135308E9
:1006A000831203178C0071248312031354088312DE
:1006B00003178C0071248312031355088312031748
:1006C0008C007124831203135608831203178C00C5
:1006D0007124831203135708831203178C007124AB
:1006E00083120313B0243B24AA2400290808F039FC
:1006F000BD003D1E8723BD1E94233D1F802B762BFE
:10070000A4240808F039BD003D1B802B08001430DC
:100710004F02031D902B1430CF00A823A123080003
:10072000CF0AA823A123080001304F02031D9D2BEF
:100730000130CF00A823A1230800CF03A823A123C1
:1007400008000808F039F03A031DA12BA424080082
:10075000CA30E4224F08A300A401F821DC01DC1513
:1007600049220800B3245230F8226130F822743054
:10077000F8226530F8222030F8220800B6245330E1
:10078000F8227430F8226530F8227030F8222030D8
:10079000F8227330F8226930F8227A30F822653076
:1007A000F8222030F82208008530E4223030F82288
:1007B0003E30F8223630F8223330F82208008530F7
:1007C000E4223630F8223430F8223E30F82231303C
:1007D000F8223230F8223730F82208008530E4223F
:1007E0003130F8223230F8223830F8223E30F82208
:1007F0003230F8223530F8223530F82208008530C2
:10080000E4223230F8223530F8223630F8223E30F9
:10081000F8223530F8223130F8223130F822080041
:100820008530E4223530F8223130F8223230F82297
:100830003E30F8223130F8223030F8223030F822C1
:100840003030F8220800B0248330E4225330F822FC
:100850006530F8227430F8227530F8227030F822B2
:100860002030F8224D30F8226F30F8226430F82220
:100870006530F8220800B024B3242030F82220305C
:10088000F8222030F8225330F8224130F822563036
:10089000F8224530F8224430F8220800B6244130CE
:1008A000F8227530F8227830F8222030F8224F30C4
:1008B000F8227530F8227430F8227030F822753042
:1008C000F8227430F8222030F8222108303EF82235
:1008D0000800831603178C130C14831203178D0A58
:1008E0000800831603178C130C1555308D00AA30A1
:1008F0008D008C148C187A2C0C11831203178D0A1E
:10090000831203130800FA30A90000000000000061
:100910000000000000000000A90B852C08008324C3
:10092000832408001430AA008324AA0B942C080006
:100930003C30AA008324AA0B9A2C08000A30AB0092
:10094000A424AB0BA02C0800C830AA008324AA0B57
:10095000A62C08001430AB00A424AB0BAC2C080070
:100960000130E42208008030E4220800C030E42294
:100970000800B024B324C5225230F8224130F822B6
:100980004D30F8225530F8222030F8225630F82227
:100990003130F8222E30F8223030F8222030F82280
:1009A0002830F8226330F8222930F822B624433068
:1009B000F8227530F8226D30F8226230F822723059
:1009C000F8226930F8226130F8222030F8224430D1
:1009D000F8226530F8227330F8226930F822673047
:1009E000F8226E30F8227330F8220800B024B324C5
:1009F000C5224730F8223330F8225230F8224F30E7
:100A0000F8224F30F8222030F8222630F822203009
:100A1000F8224730F8223430F8224730F822583094
:080A2000F8224F30F822080013
:02400E00723FFF
:0A4200000100020004000800100095
:00000001FF
